:020000040000FA
:10000000000000000328FF238316900008308500BD
:10001000843081009F018B01831207309900850194
:100020008101A001A1016400632020080739820733
:100030002B2832283928402847284E2855285C2864
:100040002008073982075C2855284E284728402871
:10005000392832282B288316083085008312203057
:100060008500132883160830850083121730850019
:100070001328831608308500831202308500132868
:1000800083160830850083123530850013288316C7
:100090000830850083120430850013288316083049
:1000A00085008312333085001328831608308500BD
:1000B00083120130850013288316083085008312CF
:1000C0003630850013282108033982076A286F28F3
:1000D00075286F2885190034A10AA00A0034851DEF
:1000E000003481010B11A10A00340B1D7928A101F4
:0800F0000034851DA10300345A
:1006600045344C3445344334543452344F344E348E
:1006700049344334203442344534413443344F34D4
:100680004E342034503449344334203431343234FD
:1006900046343634373435342034423459342034F7
:1006A00044345234203452342E34203445345234BD
:1006B0004C34493443344834203445344934443488
:1006C000203443344F34523450342E3420344634A2
:1006D000453442342E3420343234303430343834DB
:02400E008C3FE5
:00000001FF
